:100000000C9434000C94E703189500001895000038
:10001000189500000C94BA0218950000189500007D
:10002000189500001895000018950000189500001C
:10003000189500000C94A503189500001895000071
:1000400018950000189500001895000018950000FC
:1000500018950000189500001895000018950000EC
:1000600018950000189500008FEF8DBFC0EEE8EDE9
:100070004E2E84E08EBFD4E0F4E05F2EEEEFF3E08E
:10008000A0E0B1E0A89584B7082E877F84BF88E1FF
:100090009927809360009093600088278D93319713
:1000A000E9F70E94EA046624229A2A9A569A579AF5
:1000B0005F9824982C9A55985D9A259A209A529880
:1000C00021985398549880E08093800082E0809338
:1000D000810088E180936D00809169008C7F82604F
:1000E00080936900E89AE09ADA9AB09A8CE00E94CC
:1000F00038050E94DF0480E080930101E2E0F0E037
:10010000A6E1B1E094E00E94C00640E65AEE60E04D
:1001100070E0A6E1B1E00D911D912D913C910E94FE
:100120003A061CF011F00C9497000C94A10000E02A
:1001300010E020E030E0A6E1B1E00D931D932D9397
:100140003C9300E010E020E030E0AAE1B1E00D9344
:100150001D932D933C9300E010E020E030E0A2E1FD
:10016000B1E00D931D932D933C935E9A8AEF90E03E
:100170000E94BC055E988091000180688093000118
:100180000E94DD04EEE8FDE00E94D6042898A9E272
:10019000B0E08C9182FBDEF385E090E00E94BC052C
:1001A000789484B7877F84BF8FE18093600087E075
:1001B0008093600080916000886080936000A895C3
:1001C0000027A9E2B0E08C9185FB0EF401E040E04D
:1001D000041711F00C94740189E190E00E94BC05B1
:1001E0000027A9E2B0E08C9185FB0EF401E040E02D
:1001F000041711F00C947401A9E2B0E08C9185FB16
:10020000DEF7F89400910101003011F00C944A01DE
:1002100081E0809301010E94DD04E8E9FDE00E9495
:10022000D604289AE89880916F00816080936F00CF
:1002300080916800846080936800DA9AB09A80E0C8
:1002400090E0909385008093840080E08093020189
:10025000809100018F7780930001AAE1B1E00D91B8
:100260001D912D913C91A6E1B1E00D931D932D932D
:100270003C935E9A8AEF90E00E94BC055E9882E013
:1002800080938100789480910001806880930001C0
:100290000C94740180E0809301010E94E40408E062
:1002A0000E94D1040E94DD04EEE8FDE00E94D60425
:1002B000289880916F008E7F80936F0080916800F6
:1002C0008B7F80936800E89AE09A809100018F7795
:1002D00080930001A9E2B0E08C9182FBDEF385E01F
:1002E00090E00E94BC057894A8950091010100302F
:1002F00011F00C9463020027A0E0B1E08C9187FB21
:100300000EF401E041E0041711F00C946102A2E147
:10031000B1E00D911D912D913C9148EE53E060E0CC
:1003200070E00E94CB05AAE1B1E00D931D932D93DF
:100330003D93AAE1B1E00D911D912D913C9140E0DA
:1003400058E060E070E00E945C05AAE1B1E04D93E6
:100350005D936D937D93AAE1B1E00D911C914AE00C
:1003600050E00E948F04A6E0B1E00D931C93AAE137
:10037000B1E00D911D912D913C91A6E0B1E04D9120
:100380005D9157FB1EF46FEF7FEF02C06627772762
:100390000E943506AAE1B1E00D931D932D933D9384
:1003A000A6E0B1E00D911C91033050E0150780E00C
:1003B0000CF081E08F93A6E0B1E00D911C91073025
:1003C00050E0150781E014F009F080E09F91892347
:1003D000882311F40C940002AAE1B1E00D911D9163
:1003E0002D913C9145E050E060E070E00E943006C5
:1003F000AAE1B1E00D931D932D933D930C9430022F
:10040000A6E0B1E00D911C91083050E0150780E0A6
:100410000CF081E08F93A6E0B1E00D911C910930C2
:1004200050E0150781E014F009F080E09F918923E6
:10043000882311F40C943002AAE1B1E00D911D91D2
:100440002D913C914AE050E060E070E00E9430065F
:10045000AAE1B1E00D931D932D933D930C943002CE
:10046000A6E1B1E00D911D912D913C91AAE1B1E081
:100470004D915D916D917C910E943506AAE1B1E0AC
:100480000D931D932D933D93AEE1B1E0EAE1F1E0D0
:100490000E9450060E94E404EEE1F1E0A0ECB4E01A
:1004A0001127222705E034E00E94F2050E94C904CA
:1004B000E2EAFDE00E94D604809100018F778093EC
:1004C00000010C948C020027A0E0B1E08C9187FB26
:1004D0000EF401E041E0041711F00C948C02A9E243
:1004E000B1E0E6E1F1E00E9450060E94E404E9E296
:1004F000F1E0A0ECB4E01127222705E034E00E94EF
:10050000F2050E94C904E2EAFDE00E94D60480914F
:1005100000018F77809300010027A3E2B0E08C9167
:1005200084FB0EF401E040E0041711F00C94B802D3
:1005300089E190E00E94BC050027A3E2B0E08C9125
:1005400084FB0EF401E040E0041711F00C94B802B3
:1005500081E083B9E2E0F0E0AAE1B1E094E07BE77A
:100560000E94AF0684EF91E00E94BC0581E083B950
:100570000C94DF000F921F922F923F924F925F9246
:100580007F92AF92BF920F931F932F933F934F93FE
:100590005F936F937F938F939F93AF93BF93CF930B
:1005A000DF93EF93FF938FB78F9380916F008E7FD0
:1005B00080936F0000910201003011F00C94E8026A
:1005C00084E690E0A8E0B1E08D939C930C94220324
:1005D000013011F00C94F40282E390E0A8E0B1E065
:1005E0008D939C930C942203023011F00C94000321
:1005F00089E190E0A8E0B1E08D939C930C942203F4
:1006000000910201033081E008F480E08F930091B3
:100610000201043081E010F009F080E09F9189230D
:10062000882311F40C941C038AE090E0A8E0B1E068
:100630008D939C930C94220385E090E0A8E0B1E0B8
:100640008D939C93A3E0B1E089B18C93A4E0B1E0D9
:100650008C9183FB882780F9082FA3E0B1E08C916F
:1006600084FB882780F9482F0427A5E0B1E00C938C
:1006700000910501013011F00C945903A6E1B1E09D
:100680000D911D912D913C91A8E0B1E04D915D91AE
:1006900057FB1EF46FEF7FEF02C0662777270E949B
:1006A0003006A6E1B1E00D931D932D933D930C947C
:1006B0007203A6E1B1E00D911D912D913C91A8E04E
:1006C000B1E04D915D9157FB1EF46FEF7FEF02C0DB
:1006D000662777270E943506A6E1B1E00D931D93AA
:1006E0002D933D938091030180930401809100013B
:1006F00080688093000180E08093020180E090E0B8
:10070000909385008093840080916F008160809336
:100710006F008F918FBFFF91EF91DF91CF91BF91CC
:10072000AF919F918F917F916F915F914F913F9189
:100730002F911F910F91BF90AF907F905F904F903E
:100740003F902F901F900F9018950F921F922F920D
:100750003F924F925F927F92AF92BF920F931F93FF
:100760002F933F934F935F936F937F938F939F93B9
:10077000AF93BF93CF93DF93EF93FF938FB78F9395
:1007800000910201053010F00C94CB03A2E0B1E01F
:100790008C918F5F8C938F918FBFFF91EF91DF9141
:1007A000CF91BF91AF919F918F917F916F915F9109
:1007B0004F913F912F911F910F91BF90AF907F90DC
:1007C0005F904F903F902F901F900F9018950F9231
:1007D0001F922F923F924F925F927F92AF92BF9261
:1007E0000F931F932F933F934F935F936F937F9339
:1007F0008F939F93AF93BF93CF93DF93EF93FF9329
:100800008FB78F9380E283B95298219898E1AAE03C
:10081000B1E0983018F4392F992702C038E0985089
:100820004A9BFECF88941999089487954A99FECFE0
:100830003A95B1F78D93992361F75298219898E1F1
:10084000AEE0B1E0983018F4392F992702C038E0B3
:1008500098504A9BFECF88941999089487954A9995
:10086000FECF3A95B1F78D93992361F7AEE0B1E0F1
:100870000D911D912D913C91A2E1B1E00D931D933D
:100880002D933C93A4E1B1E00C9107FB00270EF4FB
:1008900001E041E0041711F00C946004A2E1B1E022
:1008A0000D911D912D913C9140E050E060E071E090
:1008B0000E943506A2E1B1E00D931D932D933D9367
:1008C00080910001806880930001EF93FF93E0E640
:1008D000F0E00E94B005FF91EF91E09A8F918FBFF9
:1008E000FF91EF91DF91CF91BF91AF919F918F9148
:1008F0007F916F915F914F913F912F911F910F9138
:10090000BF90AF907F905F904F903F902F901F903F
:100910000F901895F894FFCF00FC10D0089503D0E5
:100920001ED001F8F9CF0024E89457FF02C009D087
:10093000689400F80BD010F80124089502D009D073
:100940000895509540954F5F5F4F0895E89417FFC5
:100950000895009510950F5F1F4F68940895352FE7
:10096000242FE894452B11F468940895512F402FBB
:100970000027112780E1440F551F001F111F021B84
:10098000130B416018F4020F131F4E7F8A9599F7DD
:100990000895A0ECB4E08D91882311F063D0FBCFD3
:1009A000089580E25FD00A95E1F708950E94EE0570
:1009B000802D11F057D0FACF089580EC59C081E016
:1009C00057D005D080E854C080E852D0089583E025
:1009D0009927D2C08AEF90E00E94BC053D9A3C9ACC
:1009E0003B9A3A9A389A399A419885E090E00E9469
:1009F000BC05409845984498439A429A409AEF9390
:100A0000FF93E4ECF0E00E94B005FF91EF91409875
:100A1000B0D0409AEF93FF93E4ECF0E00E94B00571
:100A2000FF91EF914098A5D0409AEF93FF93E4ECAB
:100A3000F0E00E94B005FF91EF9140989AD0429863
:100A4000409AEF93FF93E4ECF0E00E94B005FF9131
:100A5000EF9140988ED088E20BD08EE009D086E0EE
:100A600007D00895419A829505D004D082D0089588
:100A70004198F9CF859510F4429A01C04298859526
:100A800010F4439A01C04398859510F4449A01C02C
:100A90004498859510F4459A01C04598409AEF9383
:100AA000FF93E4ECF0E00E94B005FF91EF914098D5
:100AB000089500FC05D0089530D005D001F8F9CF95
:100AC00037D03FD00895842F952FA62FB72FE894C5
:100AD000452B462B472B11F468940895402F512F36
:100AE000622F732F0027112722273327F0E2440FAC
:100AF000551F661F771F001F111F221F331F081B62
:100B0000190B2A0B3B0B416028F4080F191F2A1FF1
:100B10003B1F4E7FFA9559F708950024E89477FF1C
:100B200002C006D0689400F809D010F80124089596
:100B300012D04F5F5F4F6F4F7F4F0895E89437FF9C
:100B4000089500951095209530950F5F1F4F2F4FFA
:100B50003F4F68940895409550956095709508951D
:100B60003197F1F70895689462F80895E89462F86F
:100B7000089581E090E000C0EF93FF93EE27E82B0B
:100B8000E92B31F0E0EDF7E03197F1F70197D1F77C
:100B9000FF91EF9108950F921F922F92C801D901F2
:100BA000489F80014A9F90014B9F202C499F100D28
:100BB000211D321D5A9F202C589F100D211D321DC2
:100BC000599F200D311D689F200D311D699F300DEB
:100BD000789F300D2F901F900F900895C8953196F3
:100BE000002008952E2E3F2E992781918D3209F0F5
:100BF00093958823D1F79A95E22DF32D112361F077
:100C0000091718F011F0101B01C0191B28F021F072
:100C100080E28D931A95E9F780818D3219F48D93D6
:100C2000319604C0222311F08BE28D93091738F01E
:100C300031F0091B21F080E38D930A95E9F781914A
:100C40008D938823E1F7332351F0EA2FFB2F319660
:100C500033958E9182933A95E1F78EE28C930895C5
:100C6000040F151F261F371F0895041B150B260B95
:100C7000370B089504171507260737070895000F47
:100C8000111F221F331F0895009510952095309550
:100C90000F5F1F4F2F4F3F4F0895019110810EC0DE
:100CA00001911191219130810BC00191108117FFA9
:100CB00005C03FEF2FEF04C0008111272227332703
:100CC00037FF03C0E1DF8DE28D93CF93DF93CF92A7
:100CD000DF92EF92AA24BB24CC24DD24EE2440E250
:100CE000CAE0DD2755E093E38881890F87FD9F7077
:100CF00083FD907F891B89935A95A9F7C0DFAA1CB1
:100D0000BB1CCC1CDD1CEE1C4A9551F7E894EFE0AF
:100D1000FF2782910ED0EB30E0F71EF068948A2D09
:100D20000CD088278D93EF90DF90CF90DF91CF91FB
:100D30000895982F829501D0892F8F70805D26F0BD
:100D4000803309F4089568948D930895F999FECF3E
:100D5000E1BDF2BD3196089591E001C092E07B378C
:100D600051F47FB7F894F2DF8D9180BDFA9AF99A29
:100D70009A95C9F77FBF7727089591E001C092E067
:100D8000E5DFF89A80B58D939A95D1F708954D6572
:100D9000617375726520000043616C6962726174F1
:060DA0000000202000000D
:00000001FF
